:100000000C9438000C9466000C94ED000C94530092
:100010000C9453000C9453000C9453000C94530014
:100020000C9453000C9453000C9453000C94530004
:100030000C9453000C9453000C9453000C945500F2
:100040000C9453000C9453000C9453000C945300E4
:100050000C9453000C9453000C9453000C945300D4
:100060000C9453000C9453000C9453000C945300C4
:1000700011241FBECFEFD0E1DEBFCDBF12E0A0E064
:10008000B1E0ECEAFDE002C005900D92A638B107A0
:10009000D9F71EE0A6E8B2E001C01D92A23FB10769
:1000A000E1F70C9442030C9400001F920F920FB6DC
:1000B0000F9211248F93809186028F5F8093860226
:1000C0008F910F900FBE0F901F9018951F920F9257
:1000D0000FB60F9211248F939F93EF93FF93E091AC
:1000E0008702FF278091840090918500EE0FFF1F0B
:1000F000EE56FD4F91838083E0918702FF27809128
:100100008602EE53FD4F8083E0918702FF27E6527F
:10011000F14F81E08083E0918702FF2780911001F9
:10012000F695FE2FEE27F795E795E652FD4F808B6B
:10013000E0918702FF2780911101F695FE2FEE27AF
:10014000F795E795E652FD4F818BE0918702FF27F7
:1001500080911201F695FE2FEE27F795E795E6526E
:10016000FD4F828BE0918702FF2780911301F69566
:10017000FE2FEE27F795E795E652FD4F838BE09132
:100180008702FF2780911401F695FE2FEE27F79541
:10019000E795E652FD4F848BE0918702FF2780911F
:1001A0001501F695FE2FEE27F795E795E652FD4FE0
:1001B000858B809187028F5F809387028091870271
:1001C000883111F410928702FF91EF919F918F91E6
:1001D0000F900FBE0F901F9018951F920F920FB6A1
:1001E0000F9211242F933F934F935F936F937F93BD
:1001F0008F939F93EF93FF931DBA87E788B988B9D0
:100200008FEF88B986B18171E9F3E0918702FF270A
:100210008091840090918500EE0FFF1FEE56FD4FF8
:1002200091838083E0918702FF2780918602EE53BD
:10023000FD4F808386B18171E9F789E988B988B972
:1002400088B988B990B153B18FEF88B921E030E017
:1002500077E76FEF49E978B978B968B986B1817104
:10026000E9F3E0918702FF27F695FE2FEE27F79539
:10027000E795E20FF31FE752FD4F9083E09187026D
:10028000FF27F695FE2FEE27F795E795E652FD4FEF
:10029000E20FF31F508386B18171E9F748B948B97D
:1002A00048B948B990B153B168B92E5F3F4F2F3765
:1002B000310589F6E0918702FF27F695FE2FEE279C
:1002C000F795E795E85AFC4F9083E0918702FF2766
:1002D000F695FE2FEE27F795E795E75AFC4F5083EA
:1002E000E0918702FF27E652F14F32E03083209100
:1002F0008702809187028F5F8093870280918702B7
:100300008831B9F090918702809188029817C9F0DE
:10031000809189028F5F8093890280918902803168
:1003200020F43CBB83E08DBB0FC03CBB81E08DBBA8
:100330000BC01092870290918702809188029817D3
:1003400039F720938702E4CFFF91EF919F918F912E
:100350007F916F915F914F913F912F910F900FBEC1
:100360000F901F9018958F708A3018F0895C99272C
:100370000895805D9927089560E070E0809185027E
:100380008F7E8093850220E030E040E050E0809155
:1003900085028BB92F5F3F4F4F4F5F4F203888E367
:1003A000380781E0480780E0580789F78091850287
:1003B00080618093850220E030E040E050E0809151
:1003C00085028BB92F5F3F4F4F4F5F4F203888E337
:1003D000380781E0480780E0580789F78091850257
:1003E0008F7D8093850220E030E040E050E08091F6
:1003F00085028BB92F5F3F4F4F4F5F4F203888E307
:10040000380781E0480780E0580789F78091850226
:1004100080628093850220E030E040E050E08091EF
:1004200085028BB92F5F3F4F4F4F5F4F203888E3D6
:10043000380781E0480780E0580789F780918502F6
:100440008F7B8093850220E030E040E050E0809197
:1004500085028BB92F5F3F4F4F4F5F4F203888E3A6
:10046000380781E0480780E0580789F780918502C6
:1004700080648093850220E030E040E050E080918D
:1004800085028BB92F5F3F4F4F4F5F4F203888E376
:10049000380781E0480780E0580789F76F5F7F4F92
:1004A0006430710509F06ACF0895982F80918B020E
:1004B000873028F5292F332780918B02E09179022C
:1004C000F0917A02E80FF11D8081992787FD9095C0
:1004D0002817390709F446C041E080918B02E0916A
:1004E0008302F0918402E80FF11D8081992787FD36
:1004F00090952817390709F44BC0442341F58091A2
:100500008B028F5F80938B0280918B02873080F00B
:1005100010928B0280918F02873058F48091900264
:10052000873038F5109290028091900280938F026C
:100530000895109290028091900280938F02809192
:100540008A028F5F80938A0210928E020895109221
:100550008B0280918B028093900280919002809315
:100560008F02089580918F028F5F80938F0240E009
:10057000B4CF109290028091900280938F0280916C
:100580008A028F5F80938A0281E080938E020895B1
:10059000809190028F5F80939002B1CF982F8C3220
:1005A000A1F080918B02841778F480918B02262F22
:1005B000280F312D311DF901E050FF4F90838091BC
:1005C0008B028F5F80938B02089580918A028F5FE8
:1005D00080938A0210928B020895982F8C32C9F072
:1005E00080918B028417A0F480918B02262F280F14
:1005F000312D311DF901E050FF4F908380918B0226
:100600008F5F80938B029E3219F481E08093910278
:10061000089580918A028F5F80938A0280918B0275
:10062000841758F580919102882381F480918B0280
:10063000262F280F312D311DF901E050FF4F8EE29A
:10064000808380918B028F5F80938B0280918B02DD
:10065000841798F4772790E380918B02FB01E80FD1
:10066000F11DE050FF4F908380918B028F5F80934C
:100670008B0280918B02841778F310929102109272
:100680008B020895CFEFD0E1DEBFCDBF11B89FEF51
:1006900092B914B895B98EE087B998B980E78AB94C
:1006A0008FE88BB982E08093810081E080936F00B6
:1006B00015BE8BE08093690083E08DBB789419B1FF
:1006C00086B19927807690709595879595958795B1
:1006D0009595879595958795111F1127111F182BB3
:1006E0000E94BC01163009F45EC3153009F458C3EA
:1006F00091E083E09093C5008093C40088E18093EB
:10070000C10086E08093C200A0916F02B091700298
:100710008C91882369F0FD0131968091C00085FF9E
:10072000FCCF8C918093C600DF0181918823A9F7CB
:10073000FF248091C00087FD56C090918702809170
:1007400088029817B1F3E0918802FF27E652F14F33
:100750008081813009F467C0E0918802FF27E6526A
:10076000F14F8081823029F780918C0290918D0227
:10077000892B09F47DC180918C0290918D020197A3
:1007800009F437C280918C0290918D02029708F48F
:10079000D9C180918C0290918D028151914008F0D5
:1007A000D1C18091C00085FFC4CFE0918C02F0914F
:1007B0008D02EC5BFE4F80818093C600E0918C023D
:1007C000F0918D02EC5BFE4F8081F82680918C02C7
:1007D00090918D02019690938D0280938C0280916E
:1007E000C00087FFAACF9091C60080918A0288231B
:1007F00009F4D0C080918E02882309F0B6C08091A0
:100800008A02853009F447C2863008F033C282304C
:1008100009F48FC2833008F081C2813009F4BAC272
:1008200010928A028ACF80918C0290918D02892B3E
:1008300009F4B4C080918C0290918D02892BD1F083
:1008400080918C0290918D024197A0F48091C0001C
:1008500085FF6FCFE0918C02F0918D02E150FF4F48
:1008600080818093C600E0918C02F0918D02E1506E
:10087000FF4FAACF80918C0290918D02419770F129
:1008800080918C0290918D02479740F58091C00035
:1008900085FF4FCF809188029927E0918C02F091DB
:1008A0008D029695982F882797958795E80FF91FC1
:1008B000E752FD4F80818093C6008091880299277E
:1008C000E0918C02F0918D029695982F882797954C
:1008D0008795E80FF91FE752FD4F76CF80918C0284
:1008E00090918D02479740F080918C0290918D02FB
:1008F0008634910508F4AACF80918C0290918D02E4
:100900008634910509F460C180918C0290918D022A
:100910008734910509F4C5C180918C0290918D02B4
:100920008834910509F4C3C180918C0290918D02A5
:100930008934910509F4CCC180918502806480934B
:100940008502809185028BB910928D0210928C02E3
:10095000809188028F5F809388028091880288311D
:1009600009F406C283E08DBBE4CE80918A02853013
:1009700059F0863008F06CC1823031F0833008F0D5
:10098000C1C1813009F04CCF40E060E0892F0E9466
:10099000CE02D3CE892F0E945502CFCE8091850200
:1009A0008F7B80938502809185028BB9E0918802CC
:1009B000FF27EE53FD4F808182958F700E94B30117
:1009C00080930701E0918802FF27EE53FD4F80815D
:1009D0000E94B30180930801E0918802FF27EE0F87
:1009E000FF1FEE56FD4F80819181892F99278295B7
:1009F0008F700E94B30180930901E0918802FF2764
:100A0000EE0FFF1FEE56FD4F80819181892F9927B0
:100A10000E94B30180930A01E0918802FF27EE0F44
:100A2000FF1FEE56FD4F80819181929582958F70C8
:100A300089279F7089270E94B30180930B01E09161
:100A40008802FF27EE0FFF1FEE56FD4F8081918138
:100A50000E94B30180930C0180918C0290918D02D1
:100A6000019690938D0280938C020EE0F02E61CE61
:100A7000809185028F7E80938502809185028BB95B
:100A8000E0918802FF27EE53FD4F808182958F70A1
:100A90000E94B30180934D01E0918802FF27EE533D
:100AA000FD4F80810E94B30180934E01E091880246
:100AB000FF27EE0FFF1FEE56FD4F80819181892F9A
:100AC000992782958F700E94B30180934F01E09126
:100AD0008802FF27EE0FFF1FEE56FD4F80819181A8
:100AE000892F99270E94B30180935001E0918802D9
:100AF000FF27EE0FFF1FEE56FD4F808191819295EB
:100B000082958F7089279F7089270E94B3018093F7
:100B10005101E0918802FF27EE0FFF1FEE56FD4FB7
:100B2000808191810E94B3018093520180918C0257
:100B300090918D02019690938D0280938C022EE00D
:100B4000F22EF7CD80918C0290918D0281519140CF
:100B5000D9F180918C0290918D028251914009F4DB
:100B6000A0C080918C0290918D028351914009F434
:100B70009EC080918C0290918D028451914009F425
:100B8000A7C0809185028061809385028091850253
:100B90008BB910928D0210928C02809188028F5F27
:100BA0008093880280918802883109F4E4C08091A2
:100BB000890281508093890280918902803108F0F6
:100BC000B8CD82E08CBBCECE8091C00085FFB1CD88
:100BD0008F2D82958F700E94B3018093C600809103
:100BE0008C0290918D02019690938D0280938C02DD
:100BF000A0CDC0E0D0E004E511E0E0918802FF273D
:100C0000F695FE2FEE27F795E795E652FD4FEC0F90
:100C1000FD1F808182958F700E94B301F80180834F
:100C2000E0918802FF27F695FE2FEE27F795E795CE
:100C3000E652FD4FEC0FFD1F808121960E94B3010B
:100C4000F80181830E5F1F4FC038D105B1F6BECDCC
:100C5000883009F499CE893008F048C0863009F40C
:100C600093CE873009F0DCCD42E062E4892F0E9408
:100C7000CE0263CD873009F487CE873088F1883083
:100C800009F482CE893009F0CBCD46E067E1892FA7
:100C90000E94CE0252CD4AE06AE2892F0E94CE0223
:100CA0004CCD8091C00085FF44CD8F2D94CF809195
:100CB000C00085FF3ECD8DE08093C60080918C0200
:100CC00090918D02019690938D0280938C0231CD8C
:100CD0008091C00085FF2DCD8AE08093C60076CD3F
:100CE00041E065E3892F0E94CE0227CD893009F4C7
:100CF00045C08A3009F094CD41E060E4892F0E941C
:100D0000CE021BCD833009F43FCE843009F088CD6C
:100D100040E060E0892F0E94CE020FCD8330A1F128
:100D2000843009F07DCD41E068E2892F0E94CE0237
:100D300004CD41E06EE0892F0E94CE0280910E0129
:100D4000813469F08091150180FD09C08091850290
:100D5000806280938502809185028BB9EECC809170
:100D600085028F7D80938502809185028BB9E5CCC9
:100D700010928802F7CD1092880219CF48E067E3FD
:100D8000892F0E94ED02D9CC49E06EE1892F0E94A3
:100D9000CE02D3CC46E060E1892F0E94CE02CDCCBA
:0C0DA00090E080E4A7CC90E081E8A4CCB7
:100DAC0024424C5345432C3030303030302C2D2CD9
:100DBC003030303030302C3030303030302C30302F
:100DCC0030302E303030302C4E2C30303030302E05
:100DDC00303030302C452C30303030303030302CFE
:100DEC004D2C30302A0024424C5345512C3030309D
:100DFC003030302C303030303030303030303030EB
:100E0C0030303030303030303030303030303030D6
:100E1C0030303030303030303030303030303030C6
:100E2C0030303030303030303030303030303030B6
:100E3C0030303030303030303030303030303030A6
:100E4C003030303030303030303030303030303096
:100E5C003030303030303030303030303030303086
:100E6C003030303030303030303030303030303076
:100E7C003030303030303030303030303030303066
:100E8C003030303030303030303030303030303056
:100E9C003030303030303030303030303030303046
:100EAC003030303030303030303030303030303036
:100EBC003030303030303030303030303030303026
:100ECC003030303030303030303030303030303016
:100EDC003030303030303030303030303030303006
:100EEC0030303030303030303030303030303030F6
:100EFC00303030302A000D0A4669726D77617265A8
:100F0C002056657273696F6E3A2032340D0A0056A2
:100F1C0002244750524D432C00710224475047473E
:060F2C00412C007B02FFD6
:00000001FF
